:10000000B86D0010B5010000B9010000BB0100008F
:10001000BD010000BF010000C1010000E287FFEF49
:10002000000000000000000000000000C30100000C
:10003000C501000000000000C7010000C901000068
:10004000CB010000CB010000CB010000CB01000080
:10005000CB010000CB010000CB010000CB01000070
:10006000CB010000CB010000CB010000CB01000060
:10007000CB010000CB010000CB010000CB01000050
:10008000CB010000CB010000CB010000CB01000040
:10009000CB010000CB010000CB010000CB01000030
:1000A000D7260000CB010000CB010000CB010000EF
:1000B000CB010000CB010000CB010000CB01000010
:1000C000CB010000CB010000CB01000000F002F8E2
:1000D00000F046F80AA090E8000C82448344AAF19C
:1000E0000107DA4501D100F03BF8AFF2090EBAE89A
:1000F0000F0013F0010F18BFFB1A43F0010318475C
:10010000CC560000EC560000103A24BF78C878C1E5
:10011000FAD8520724BF30C830C144BF04680C600D
:10012000704700000023002400250026103A28BF55
:1001300078C1FBD8520728BF30C148BF0B60704759
:10014000642904F03785732904F0F786002070478E
:100150001FB59DE8030004F029FE1FBD10B510BDBA
:1001600004F03CFF1146FFF7F3FF00F018FB04F02A
:100170005AFF03B4FFF7F2FF03BC04F08BFF00004B
:10018000D0F800D0D0F804F070B50023084D0AE094
:10019000CE5C04885B1C86EA14269BB235F8166098
:1001A00086EA04240480521E92B2F1D270BD00008F
:1001B000E051000008480047FEE7FEE7FEE7FEE7E3
:1001C000FEE7FEE7FEE7FEE7FEE7FEE70348044939
:1001D000044A054B70470000CD000000B81D001018
:1001E000B86D0010B85D0010B85D0010064802211F
:1001F00041600021016741610B22C260C16301219E
:10020000416000207047000000000940EFF31080BB
:1002100010F0010F72B64FF080404FF000020270F4
:100220004FF0AA0303724FF05504047202614FF0BD
:10023000FF0242604FF0030202700372047200D1A9
:1002400062B6FEE770B5284C607820B30026274DD3
:10025000012810D002280DD1A8686168401A2449ED
:10026000884215D32348406B400011D5012002F08D
:100270000CF9667070BDA8686168401A1E49884212
:10028000F8D3002002F001F9A868606002206070D5
:1002900026700C2005E020780028EBD1012020708A
:1002A0000D20BDE8704001F04FB9002802D10E4981
:1002B00001204870704710B501F004FE0A49002083
:1002C000487010BD084801214170084989684160A3
:1002D000704770477047022803D0032803D100F00D
:1002E00016BE00F031BE7047080100100000094042
:1002F000A086010000C0092040420F00FFFFFFFF61
:100300001948042101610721016000214161416216
:1003100002214160C168C906FCD400E08168C1685F
:100320004907FBD4002070470F498860C868C006A1
:10033000FCD48868704700B50B46024604E000BF55
:1003400012F8010BFFF7F0FF5B1EF9D200BD00B5FC
:100350000B46024604E00020FFF7E6FF02F8010B1F
:100360005B1EF8D200BD00000080084070B5064654
:1003700004F002FD056806F10B0020F00704B4420A
:100380009CBF002070BD2B466A68BAB11068A042BD
:1003900010D304F1080188423CBF5068586007D36D
:1003A0005168101941601168091B016058601460A0
:1003B000101D70BD13465268002AE7D12146284619
:1003C00004F0E0FC0028DED170BD00000FB41CB5C5
:1003D0000C0007AA009001D02044401E074B7B442C
:1003E00069460190069804F076FD002C03D069461A
:1003F000002004F083FD1CBC5DF814FB254B0000BD
:10040000704770474D0B000010B5FE49486D000560
:100410000CD4FD4A906843F698239468241A9C42B1
:10042000FBD3486D000501D4012010BD052001F06B
:100430008BF8002010BD70B5F34CA668042001F0C5
:1004400083F8F24D03E000BFFFF7DEFF48B1A0687C
:10045000801BA842F8D308E0FFF7D6FF08B10120BF
:1004600070BDA068801BA842F6D3002070BD2DE9A6
:10047000F041092001F068F8E54800264FF47A774A
:100480000670C821384601F015FADF4CA06842F228
:100490001075A168091AA942FBD3C821384601F09A
:1004A00009FAA068A168091AA942FBD3C8213846F5
:1004B00001F000FAD748022186708171C670BDE84C
:1004C000F0818AB04FF0000946208DF814008DF8B5
:1004D00017903D20CA4600905446CFA3CFA20A21D0
:1004E00005A8FFF773FFCF4908684FF6FF021040D9
:1004F000CD4A40F4807010430860CC48CD49D04DBF
:100500000460CB480068A0F56C50FF380860CA4909
:1005100000F5E0500860C949400A0860F8202870DA
:10052000FF206870A87001F05DF9BA4CC54A002040
:1005300094F9051052F821102A1802F580520B5C2C
:10054000401C82F800386028F6D34FF4E175294644
:1005500040F2491001F0AEF9294640F29F1001F037
:10056000A9F94FF4005BDFF8E0825D46207808B11E
:10057000FFF768FEA07928B1012818D0207800285C
:1005800079D0FCE00A2000F0DFFF00F017FE10B188
:10059000FFF76DFFEAE70120A0715D4684F803A034
:1005A000062000F0D1FF0A2000F0CEFFDEE719227E
:1005B0002946A54800F0C2FD98F8180000287CD014
:1005C00098F80000062873D2DFE800F072030B46AB
:1005D000464940F2044000880290D8F80410814255
:1005E00066D098F809104FF00109404601295FD103
:1005F000D0F80A1019B995498969C0F80A1000267F
:10060000804617E0072000F09FFFD7F80E00B8469D
:10061000871B402F00D94027A9193A468C48193129
:1006200000F08CFDD8F80A003A463044884900F0C2
:10063000F9FE3E44D8F80E004746B042E2D8397879
:10064000012935D14FF0E0220906C2F88011D7F810
:100650000A0000F015FF2BE04FF001092BE098F89D
:1006600009104FF00109032925D17149794A002663
:100670000B68136017E07BE0072000F065FFD7F8F8
:100680000E00871B402F00D94027A9193A46704811
:10069000193100F053FD66483A46006881196C48EC
:1006A00000F03BFD3E44D8F80E004746B042E3D888
:1006B00098F8180008B1464600E01CE098F80800D9
:1006C000C00613D56349012202A8C1F800B005F1A4
:1006D0001801CDF808A000F011FD307820B1C82134
:1006E0004FF47A7001F0E6F8307E20B1307A80075E
:1006F00001D5FFF78BFDD8F80E001B350544524895
:1007000000F050FD30B30220A07141485D4680F8F2
:1007100000A00B2000F018FFB9F1000F1AD03A4AE0
:100720004FF00009916842F2107093685B1A83429F
:10073000FBD34FF42F714FF47A7001F0BBF83148BE
:10074000406D400502D50020099001E0099808B9E4
:10075000FFF75CFDE078401CC0B2E0700C2802D3CB
:100760000120A07014E7A07800283FF413AF0FE732
:100770000120207001F0C8FE012001F086FE24480F
:1007800000780028F1D0002105A800F029FC0028FD
:10079000EBD084F806A05D4684F803A0E6E61D4C85
:1007A0000026FF202660A680A671607100F06CFF15
:1007B00001F0AEF8FFF71AFD00F08CFE002000F00B
:1007C000C3FEFFF79DFDFFF71FFEC8B1042000F038
:1007D000BBFE0C4F786D0C4D000541D4FFF72BFE8E
:1007E00070B1FFF728FE58B1FFF725FE40B1042095
:1007F00000F0AAFEA86805497A6D120530D42BE0F6
:1008000036E0000000C009200000094080841E007E
:1008100068000010BC00001046000000257325642D
:10082000000000000CED00E00000FA05AC00001034
:10083000B80000109C0000109400001098000010F8
:1008400035010010600000101C0100102055000050
:10085000AD1B0010B0000010AA68121A8A42CBD358
:10086000A86842F21071AA68121A8A42FBD3667114
:1008700000F036FC00F0A2FC80B100F008FE68B188
:10088000022000F061FE94F90500401C03D10D48E0
:10089000806900F0F5FD0120607004E0022000F0A6
:1008A00053FE66706671FFF7AFFD40B14021064808
:1008B00004F03DFA4022D101034800F02EFCFFF77E
:1008C00000FE000020550000AD1B00102DE9F04790
:1008D000FE4A00234FF40077156A4FF4FF79C5F301
:1008E0000724DFF8ECA34FF4E05CDFF8E883FA4E6E
:1008F00025E0B84216D213280CD014280CD0484555
:100900000CD0A0F58072FF3A0AD03E2813D81AF80E
:10091000002011E0EAB20FE022460DE055220BE084
:10092000AA2209E0604506D208EB0002A2F5805237
:1009300092F8002E00E00022F254401C5B1C8B4217
:10094000D7D3BDE8F08770B5E04D2C6B402C00D9B3
:100950004024E86AE96902198A4202D90C1A042182
:1009600069702146FFF7B2FF2246DB49822001F081
:1009700088FEE86A2044E862286B011BD748296397
:100980008268A2EB0402826005D06978022901D056
:100990000021017370BD03216970F9E7CF4910B5DB
:1009A000CF4808600D22822001F06BFEC749052068
:1009B000487010BD70B50D46CA49496D490521D42E
:1009C000B0F5007F1ED3C849C04CB0F5E05F1AD225
:1009D0008A68A369D21AC54B9A4204D38968A16177
:1009E000002161606161BD4900235F39B94A07E0B8
:1009F000C4181444CE5CA4F580545B1C84F8006ECB
:100A0000AB42F5D370BD626922B98A68A2618A6877
:100A10006261A060B64A5279002AF3D18A6863699C
:100A2000D21AB44B9A421CD2B34B01221A708A6874
:100A3000A26189686161A168401A6168884203D92E
:100A4000616A884200D26060062000F07DFD616826
:100A50002A46BDE87040A14801F500515F3800F01A
:100A60005CBBBDE870400C2000F06EBD10B5974C2B
:100A7000A178E06A4218E1698A4206D9081AA07092
:100A800005206070022001F0B7FDA178E06AFFF751
:100A900091FFA178E06A0844E062206B421A8F4817
:100AA00022638368A3EB0101816002D0617805298C
:100AB00004D100210173BDE810406FE710BD2DE99E
:100AC000F041824CA178E06A4218E1698A4206D975
:100AD000081AA07005206070022001F08DFD7F4D86
:100AE0000021A0787C4B5F3DE26A08E056186F5CFD
:100AF0009E5DBE4202D00021A16202E0491C8142FB
:100B0000F4D31118E162216B0A1A744922638B68CD
:100B1000A3EB0000886002D06078052808D1A06AA5
:100B200020B100200873BDE8F04137E70120F9E764
:100B3000BDE8F081694810B51F38D0F81110027D6A
:100B400009BA21F0FF011143604A4902D162C18A0A
:100B500049BA49021163806888420CD0822001F0B2
:100B60004BFD022001F048FD5C4902200873FFF7AD
:100B700015FF002010BD012010BD70B55748574D1E
:100B80001F380224816829B1007B000607D40220A7
:100B900001F032FD2C73FFF701FF002070BD012032
:100BA00070BD10B54D48494C1F388068A178884207
:100BB00000D2A0704949A2785F39822001F061FD1E
:100BC000032060704548A2788168891A81600021FD
:100BD000017310BD414810B51F38816839B1007BE1
:100BE000000601D5822000E0022001F005FD3B490E
:100BF00000200873BDE81040D0E610B5FFF7BDFF38
:100C000000281FD0354870215F3802220170002172
:100C100041708270C1700171417181710A22C2718B
:100C2000017241728172C1723022027301224273D9
:100C30008173C17301744174244912208870BDE826
:100C40001040AEE710BD1CB5FFF797FF00286AD033
:100C50002A480A2206210388684600F025FA1F4820
:100C600000225F3880230270437082700121C170BE
:100C70002021017143718271C2714122027254229A
:100C800042724F2282724C22C2720173417381738D
:100C9000C173462202745023437472238374692300
:100CA000C3746E230375742343758175C2756C22FA
:100CB000027661224276732282766822C2760177BA
:100CC00041778177C1779DF8011019E07800001015
:100CD000E054000035010010AD1B0010941B001003
:100CE0005553425300C0092000000940A08601006E
:100CF000BC00001020A107006800001004040000E0
:100D000080F820109DF8021080F821109DF8031043
:100D100080F822109DF8041080F82310DE4924206A
:100D20008870FFF73EFF1CBD10B5FFF726FF0028B7
:100D30000CD0DA4803210170002141708170C1702C
:100D4000D54904208870BDE810402AE710BD10B5D1
:100D5000FFF713FF002810D0D048002106220170B1
:100D600042708170C170017141718171C171CA4954
:100D700008208870BDE8104013E710BD10B5FFF7DC
:100D8000FCFE002815D0C44AC448116A491E0B0E47
:100D900003700B0C43700B0A8370C170002101714A
:100DA000417102238371C17108209070BDE8104029
:100DB000F7E610BD10B5FFF7E0FE002819D0B748E0
:100DC0000021B54B0170417081700822C2701A6A0F
:100DD000140E0471140C4471140A8471C27102223D
:100DE000027241728272C1720C209870BDE810408C
:100DF000D7E610BD2DE9F041A74DA84C0021A878F9
:100E00004034A64A02E0535C6354491C03468142C5
:100E1000F9D31F2B72D12068A14988426ED19F4E11
:100E200060685F364FF001087060A068B060607B5A
:100E300018B9A07B08B1102802D986F80C8059E0B7
:100E4000E07B1E28F9D00FDC12282ED005DC48B339
:100E50000328F2D1BDE8F041CFE61528EDD01A28DD
:100E6000EBD1BDE8F0415FE702272A2828D010DC4B
:100E700023281DD025281ED02828DED1FFF75AFEB2
:100E8000002826D0207B000618D56F70BDE8F04101
:100E900059E52F281ED05528CFD05A28CDD1BDE8EE
:100EA000F04154E7BDE8F04194E6BDE8F041CAE600
:100EB000BDE8F0417EE7BDE8F0415FE7022016E0C3
:100EC000FFF738FE002804D0207B00060ED485F8FA
:100ED00001802DE6FFF72EFE0028FAD0207B0006C9
:100EE00004D485F80180C5F8288021E6822001F02D
:100EF00083FB3773BDE8F04150E5FFE7822001F046
:100F00007BFB022001F078FB0620687010E6624847
:100F100010B54178022908D003290ED004290FD03A
:100F2000052901D10021417010BD5C484030C07BD3
:100F30002828F9D1BDE8104005E5BDE810402DE5B1
:100F4000822001F059FBF8E710B55449022001F066
:100F500067FB51498870487858B101280CD00220AD
:100F600001F04AFB4D4902205F310873BDE8104093
:100F700014E5BDE810403DE748484030C07B2A28D2
:100F800004D02F2805D1BDE8104098E5BDE81040F9
:100F90006CE510BDFFB50246002002EB420501469C
:100FA0004FF440566C4603AA6B1844F82130B34204
:100FB00002DD002004B0F0BD3A4F07EB6307DB070A
:100FC0003F78575401D03B095354535C8F0003F0D2
:100FD0000F035354BB40491C18440329E4DBE9E7E1
:100FE000F0B506460020034602462E4C4FF400772B
:100FF00000E05B1CF55C45B102EB030CA4440CF56E
:10100000805C9CF800C8AC45F3D0032B3FD302F5BD
:10101000C0502044037F457FC67F03EB0523857FB7
:101020002D0405EB06652B4451EA03052BD021B9AD
:101030001949496840318B4225D8184B00216C333F
:101040005518254405F5805595F800585D54491C00
:101050000C29F5D3817EC27E01EB0221027D407D09
:10106000120402EB00600C182046FFF793FF40F6D5
:10107000F57501E0FFF78EFFC11EA942FAD3A0F576
:101080007061FF3901D00020F0BD2046F0BD203254
:10109000BA42AFD3F0BD000078000010351B00103D
:1010A0005553424335010010FFB5ACA60446E1CECE
:1010B0008DE8E100022902DA002004B0F0BD6018DA
:1010C000002100F8011D6946B3FBF2F502FB15355E
:1010D000B3FBF2F34D5D00F8015DA042F4D8ECE7FC
:1010E00010B503F024FC03F00EFCA0494FF40052AD
:1010F000C1E90020A0F5F420886010BD70B503465A
:1011000008468D189949002449688D4200D9881AEB
:10111000194603F05BFC204670BDF8B51446934EAB
:101120000A460B19716800258B4200D90A1B034639
:101130000094306803F075FC2846F8BD10B50B46E6
:1011400001460024184603F015FC204610BD2DE989
:10115000FC410746002090460E46ADF800000446CC
:101160000EE0351B402D00D9402539192A4680480C
:10117000FFF7E4FFAAB27E496846FFF705F82C4462
:10118000B442EED33919424601A8FFF7D7FFBDF8A4
:101190000000BDF80410884202D10120BDE8FC81A6
:1011A0000020FBE70021425C12B9491C1829FAD340
:1011B000182901D000207047012070472DE9F04127
:1011C0006A4C00270C3488B0A770E770DFF8A48160
:1011D0004FF40056277101251922314601A8FFF767
:1011E000ADFF022216213046FFF7B1FF00287DD067
:1011F000DDF81210022206F11900FFF7A8FF0028FF
:1012000074D09DF8040006282AD2DFE800F02A03F3
:10121000032A2A1CD8F87410DDF80E30491C8B42C2
:101220001ED2D8F87420DDF80E30D21ADDF8123054
:10123000521C9A4214D3DDF80E20DDF812301A4405
:101240008A420DD80DE0DDF81210B1F5F42F00D967
:10125000A570DDF81610C1F30B41B1F5087F00D081
:10126000A570012803D0022801D0052839D1022217
:1012700006F21D4168460097FFF760FF009902984B
:1012800089B2884200D0A570012206F22541684645
:101290000097FFF753FF0099BDF80500C9B28842D7
:1012A00000D0A5709DF8040002281AD1042206F28D
:1012B000494168460097FFF741FFDDF816000099A5
:1012C000884200D0A570012206F24D416846009781
:1012D000FFF734FF00989DF80710C0B2814200D09C
:1012E000A5709DF81C00401EFE2800E01FE000D203
:1012F000A570BDF80500A0F57F41FF3901D03D285C
:1013000002D19DF8070020B901A8FFF74BFF00B9F3
:10131000A570DDF812001B36064401A8FFF742FF56
:1013200030B1E07880B1217988420DD012E0A5700B
:101330009DF81C0010B92079401C2071E078401CF9
:10134000C0B2E0700C2801D3A57003E0A07800289B
:101350003FF442AFA07808B0BDE8F08130313233BD
:10136000343536373839414243444546B0000010E1
:10137000AD1B0010985500004F4A104710B572B6CB
:1013800033244E4B10C307C34D484FF47A710068A5
:10139000B0FBF1F01860191D4848FFF7EDFF62B689
:1013A00010BD464A32231360C2E9010144484FF49C
:1013B0007A710068B0FBF1F0D06002F114011046C0
:1013C000DAE73E4A34231360C2E901013C484FF496
:1013D0007A710068B0FBF1F0D06002F114011046A0
:1013E000CAE710B572B60624364900BF51F824206A
:1013F000824212D93349783951F82410814207D1F9
:1014000021460846FFF7CDFF21460846FFF7D9FFE2
:1014100021460846FFF7C5FF02E0641C1D2CE5D9F4
:1014200062B610BD2DE9F041274C236803B9206056
:10143000224D00202835636803E00F5C1E18401C15
:10144000AF559042F9D398184FF480766060B0425F
:1014500013D12068FFF7C5FF184D1435286800B177
:10146000FEE71649324628312068FFF787FF2868D3
:1014700000B1FEE70020606020600020BDE8F08140
:1014800072B61249124A01401160FEF779BE46F267
:10149000044000210088A0F51942993A0AD04FF47F
:1014A000C0404FF4002208C890421944FBD309B150
:1014B0000020704701207047F11FFF1FF01B001034
:1014C000D800001098550000C400001080FFFF1FD6
:1014D00008ED00E0002070476949C20702D04FF4D0
:1014E00080028A61800702D54FF4001088610020D5
:1014F00070476349C20702D04FF48002CA61800777
:1015000002D54FF40010C86100207047014600204A
:101510005B4ACB0703D053695B0200D501208907E2
:1015200004D55169890201D540F00200704710B519
:101530000446FFF7EBFF0346FFF7DBFF24EA030057
:10154000FFF7CAFF002010BD70B54E4B50B159686F
:10155000042403250226052907D2DFE801F0072B22
:101560004A718E0000205860986070BD042807D032
:10157000052809D0012402287AD0012808D00FE0DC
:101580000320FFF7B6FF46E0BDE870400120B0E75A
:101590000320FFF7AEFF0BE0FFF79EFF5C6070BD1E
:1015A0000E28FCD10320FFF7A4FF0220FFF794FFD1
:1015B0000120F1E706280AD0032810D00A2813D00A
:1015C000092811D00D280FD00C28D9D070BD0320C8
:1015D000FFF78FFF0220FFF77FFF5E6070BD0320E3
:1015E000FFF787FF012027E00320FFF782FF02209B
:1015F00012E0062813D00A281AD00928C8D00C28CF
:10160000BED00D28F0D00F28E8D10320FFF771FFDE
:101610000220FFF761FF0120BDE870405CE7986899
:1016200010F01F0F00F101009860D7D102201BE0DD
:101630000320FFF75EFF0220FFF74EFF5D6070BDE5
:10164000072806D00A289BD00B2811D009289FD044
:1016500070BD0220FFF74DFF986810F03F0F00F1BA
:1016600001009860F4D10120BDE870405FE7FFE71A
:101670000320FFF73EFF02208EE70628A7D08FE762
:1016800000C00920CC0000104F4810B52021C0F840
:10169000A01100BFD0F8A0114906FBD50521C0F864
:1016A00004114FF04472C0F8A8214FF48062C0F8D2
:1016B000AC210122C0F80C210B23C0F88430C0F803
:1016C0008020AA22C0F88C205523C0F88C3000BF9F
:1016D000D0F888406401FBD50324C0F88040C0F8EE
:1016E0008C20C0F88C30C0F808113849C0F8C410FC
:1016F0000021C0F8C811D0F888106FEA11618A077C
:101700003349D0F80C2102F0030207D07AB3012A42
:1017100044D0022A47D0032A4ED13AE02AB1012A06
:1017200013D0022A24D0032A46D1D0F88820D0F83A
:101730000431C2F30742DBB2521C5B1C5A43D0F89F
:101740008830244CC3F30E030EE0D0F88820D0F884
:101750000431C2F30742DBB2521C5B1C5A43D0F87F
:1017600088301D4CC3F30E035B1C634321E010E083
:10177000D0F88820D0F80431C2F30742DBB2521C03
:101780005B1C5A43D0F888304FF47A44C3F30E03FD
:10179000EAE7D0F80421114BD2B209E0D0F80421D5
:1017A0000F4BD2B204E0D0F804214FF4FA43D2B286
:1017B000521CB3FBF2F20A60016821F4704141F45B
:1017C0000051016010BD000000C00F40DE96E883AC
:1017D000D800001000127A0000366E0100093D00AA
:1017E000001BB700434900200867C86010224A6107
:1017F0008861C022CA6340498A684049C1E9002023
:101800003F4908603F49086078463F49086000202A
:1018100070472DE9F04341F288320023384C394DAE
:10182000394E904208D8642800D228B942F210728A
:10183000914201D8052907D28620206078462B6086
:1018400030608620BDE8F083DFF8AC90D9F808203E
:10185000DFF8A880D8F80070D21BD8F8047007EB26
:10186000470CCCEBC717B2EBC70F06D205202060A0
:1018700078462B6030600520E4E71E4A0227576057
:10188000D2F83CC00CF0FD0CC2F83CC040B1DFF80F
:101890007CC0BCFBF0F04010D0615760012050606C
:1018A000D9F80800C8E90001236078462B60306051
:1018B0000020C7E770B5114C00250E466560FFF7A4
:1018C000A8FF0F49000601D5086870BD0A4B06EB5A
:1018D00046022068C2EBC6129E68361AB6EBC20FEB
:1018E000FAD3044802224260C26B02F0FD02C263D6
:1018F0006560E9E70080004000000940DC0000105E
:101900006C0000107000001074000010001BB70085
:10191000F0B5FF4800218162816821F44021816097
:10192000816C21F4402141F400218164F949421580
:10193000CA630A6A42F400720A62426A22F0407282
:1019400042F000724262426E22F0407242F0007237
:101950004266426A22F0406242F000624262426E97
:1019600022F0406242F000624266C26842F0407279
:10197000C260C26C22F0407242F00072C26402691E
:1019800022F440520261026D22F4405242F40052AD
:10199000026540238B650A6C42F040020A640269CA
:1019A00022F003020261026D42F00302026501228D
:1019B000CA650A6C42F001020A64026922F00C0254
:1019C0000261026D42F00C0202650222CA650A6CD5
:1019D00042F002020A64026922F030020261026DE2
:1019E00042F0300202650422CA650A6C42F0040229
:1019F0000A64026922F0C0020261026D42F0C00274
:101A000002650822CA650A6C42F008020A6402698B
:101A100022F440720261026D42F4407202651024A9
:101A2000CC650A6C42F010020A64026922F440623A
:101A30000261026D42F4406202652025CD650A6CA8
:101A400042F020020A64026822F4404242F400425A
:101A50000260026C22F440420264026822F44022D6
:101A600042F400220260026C22F4402202644268C6
:101A700022F00C024260426C22F00C024264DA0254
:101A8000CA610A6822F400320A60426822F0300219
:101A90004260426C22F0300242F0200242641E0397
:101AA000CE610A6822F480220A60026842F4403261
:101AB0000260026C22F4403242F400320264C268D6
:101AC00042F04042C260C26C22F0404242F000420A
:101AD000C264026822F0300242F010020260026C1E
:101AE00022F0300242F020020264026822F0C002BA
:101AF00042F040020260026C22F0C00202640268FE
:101B000022F0404242F080420260026C22F04042E9
:101B100042F000420264426822F00302521C42601A
:101B2000426C22F003024264026922F4403242F421
:101B300000320261026D22F4403242F4003202654A
:101B4000026922F4402242F400220261026D22F472
:101B500040220265026822F00302921C0260026CBD
:101B600022F00302921C0264026822F00C0242F08E
:101B700008020260026C22F00C020264C26842F4A5
:101B80004032C260C26C22F4403242F40032C2647D
:101B9000C26842F44042C260C26C22F4404242F445
:101BA0000042C264C26842F44072C260C26C22F455
:101BB000407242F40072C264C26822F44052C260B1
:101BC000C26C22F44052C2641A048A630F6A47F45A
:101BD00080070F62C76827F03007C760C76C27F01F
:101BE0003007C7648E630E6A46F480260E6246682C
:101BF00026F0407646F080764660466C26F04076C9
:101C00004664466826F4400646F480064660466C04
:101C100026F440064664466846F440764660466CC4
:101C200026F440764664466846F0C0064660466C38
:101C300026F0C0064664466826F0406646F0806698
:101C40004660466C26F0406646F00066466446688C
:101C500026F0405646F080564660466C26F04056C8
:101C600046F000564664C66826F0405646F00056D8
:101C7000C660C66C46F04056C664C66926F4402667
:101C8000C661C66D46F44026C665D600CE670E6EA8
:101C900046F000760E66466826F4404646F48046D6
:101CA0004660466C26F4404646F400464664466864
:101CB00026F4403646F480364660466C26F44036BC
:101CC00046F400364664466826F4402646F48026EC
:101CD0004660466C26F4402646F400264664466874
:101CE00026F4401646F480164660466C26F44016EC
:101CF00046F400164664C66846F44026C660C66CC4
:101D000026F4402646F40026C664C66804E00000B7
:101D100000C0024000C0092026F00306C660C66C61
:101D200026F00306B61CC66496118E630E6A46F44E
:101D300080360E62066926F440060661066D26F4BA
:101D400040060665C614CE650F6C27F400670F6465
:101D5000476827F440574760476C27F4405747F4DB
:101D600000574764CA610A6842F480020A60426808
:101D700022F440624260426C22F4406242F400620B
:101D80004264DA03CA610A6842F400120A60026916
:101D900022F440120261026D22F440120265021523
:101DA000CA650F6C27F480670F64076827F44057F3
:101DB0000760076C27F440570764CB610B6823F07A
:101DC00040030B60C36823F4400343F48003C36003
:101DD000C36C23F4400343F40003C364C36823F0DB
:101DE000C003C360C36C23F0C00343F08003C3642B
:101DF0005302CB630B6A43F400230B62836823F422
:101E000040338360836C23F4403343F400338364B2
:101E100083158B630B6A43F480730B62836823F42E
:101E200040138360836C23F4401343F400138364F2
:101E3000CA630B6A43F480630B62836823F04053E8
:101E40008360836C23F0405343F000538364130199
:101E5000CB630B6A43F480430B62036823F44003B3
:101E60000360036C43F440030364CE610B6823F406
:101E700000630B60036823F440130360036C43F4B6
:101E800040130364CA610A6822F480620A6002682F
:101E900022F440620260026C22F4406202648D61AE
:101EA0000A6842F020020A60026822F4407202606E
:101EB000026C22F440720264CC61086820F01000C9
:101EC0000860F0BDFA4800214FF0011281800170D6
:101ED0004170C0E902217047F5491C31002000F033
:101EE0009FBB10B5F24C1434A288402A00D940227E
:101EF0008020216800F0C5FB216801442160A18891
:101F0000081AA08010BD10B5E94C002014342168D7
:101F100000F086FB216801442160A188081AA08096
:101F200010BD00221146802000F0ABBBE14900202B
:101F300000F076BB70B5DE48DD4D1C3005F11405B0
:101F4000007810F01F040AD0D949DA4B01F11C00C7
:101F50004A780079012C06D0022C26D109E0D44819
:101F6000001D28601DE002B3897888421DD2002040
:101F700015E000F08F04200605D504F00F064FF49D
:101F80008030B04001E00120A0400AB922070CD106
:101F90008A68024209D0C9680142E8D0012018804D
:101FA0002B60FFF79EFF012070BD002070BD024630
:101FB00070B5BF48BE4C1C30017811F01F030146BC
:101FC000498804D0012B29D0022B27D111E0012907
:101FD00024D132B1012000F0BDFAA08840F0020007
:101FE00005E0002000F0B6FAA08820F00200A080F2
:101FF00021E0007900F08F00030605D500F00F0303
:102000004FF480359D4001E00125854063782BB178
:10201000030703D0A3682B4200D009B1002070BD94
:1020200022B100F0E9FAE068284303E000F0EEFA9C
:10203000E068A843E060012070BD9D4810B51C30E9
:10204000007810F01F0F9A4800F11C00C0782AD1C8
:1020500097491431012807D001F10802022893782A
:1020600006D003281FD112E093480860122012E026
:102070009248002204E004780CB144882044521CA9
:102080009342F8D1027872B10860408803E08C482E
:102090001844086000788A88824200D98880FFF757
:1020A00020FF012010BD002010BD2DE9F84F804F0A
:1020B00000201C370090B8787D4E4FF000094FF09B
:1020C000010A4FF4803B00286BD07C4C65E06078BF
:1020D000022804D0042841D005285CD141E0617970
:1020E000B878814238D170702079B0707049002082
:1020F00011F1100101F80090401C0428FAD30125C9
:102100004FEA06080AFA05F0D8F80810084202D08B
:10211000284600F05DFAD8F808100BFA05F00842DE
:1021200003D045F0800000F053FA6D1C102DE9D368
:102130004FF00110C8E90209012000F00CFAE07923
:102140004006B8F8040002D540F0010001E020F09C
:102150000100A8F804001EE060881DE0E07800900F
:1021600019E00098B8B9A07800F08F05280604D5CA
:1021700005F00F010BFA01F001E00AFA05F0B16871
:1021800001432046B16000F0FCF9284600F016FA41
:10219000284600F027FA207804442078002896D1B9
:1021A0001FE086F8019001245546D846B16805FA2B
:1021B00004F0084202D0204600F00AFAB16808FA9A
:1021C00004F0084203D044F0800000F001FA641CDF
:1021D000102CEBD34FF00110C6E90209002000F0EB
:1021E000BAF9B8787178884202D10120BDE8F88F39
:1021F0000020FBE72DE9FC5F2D4D00273E46687867
:10220000BB46B846002871D0BA462C4C05F11C09D3
:1022100068E06078022804D0042808D005285FD13F
:1022200019E06079697888425AD0608859E0A778C7
:1022300099F80410E6784FF00008B94250D199F8A7
:102240000200B0424CD11A484FF0010A103010F889
:1022500007B0C65544E099F80410B94240D1A178BE
:1022600001F08F010191090605D5019901F00F02D6
:102270004FF4803101E0019A01219140009199F8D9
:102280000200B0421ED1A8680843A860E96800981F
:1022900081432046E96000F074F9019800F08EF95E
:1022A000019800F09FF9009948EA010818E0000041
:1022B000E4000010181D0010105600002256000007
:1022C000435600005E450BD118EA010F08D1A868FB
:1022D0008843A860E8688843E860019800F078F9CE
:1022E000207804442078002893D15046BDE8FC9F14
:1022F0002DE9F041494C0027A4F108062178A4F10A
:102300001C05082863D2DFE800F062046472626290
:102310008381FFF7E1FD2078C00900F04EF9E088E5
:10232000B0802078C0F34111F1BB61780C294AD20A
:10233000DFE801F00609490B49101A1D1F2531423B
:10234000FFF7F8FD4DE0002000E00120FFF72FFE31
:1023500050B306E010F01F0F35D1A07840F0800098
:102360002870BDE8F041DCE5FFF767FE39E00020AA
:102370002AE010F01F0F26D128481B381AE010F071
:102380001F0F20D1FFF791FE70B1FFF7CAFDBDE826
:10239000F041FDF79FBF00F01F00012813D16878BE
:1023A00010B12079A97800E00DE088420BD21B49DA
:1023B0000C39084430601CE000F01F00012802D1F5
:1023C000FFF718FFC4E7802000F016F9B780BDE8DA
:1023D000F081080608D4B0880028F8D0FFF793FDF4
:1023E000B0880028EFD0F2E7BDE8F0419EE508068E
:1023F00002D5BDE8F04174E528780106E7D500F084
:102400007F002870BDE8F04100F054B8802000E063
:102410000020BDE8F04100F0F9B800000001001014
:1024200001460007C00E090600D5401C7047DA4976
:102430001022C1F80822C1F8100200BFD1F8000232
:10244000C006FBD57047D44A1023C2F80832C2F840
:10245000100200BFD2F80002C006FBD5C2F8083255
:10246000C2F81012D2F80002C006FBD57047CA4964
:102470003022C1F80822C1F8100200BFD1F80002D2
:102480008006FBD5D1F81402704710B5040001D0C6
:10249000012000E000204FF4807141EA0041BF4874
:1024A000FFF7D1FFBE494FF000700CB1886710BD37
:1024B000C86710BD30B5BB49BB4D41EA0044214659
:1024C0002846FFF7C0FF21462846BDE83040BAE75E
:1024D000B1480021C0F848124021C0F84C12012236
:1024E000C0F84822C0F84C12D0F80012C905FBD53C
:1024F0004FF0FF31C0F83812C0F83412C0F808129B
:102500000C21C0F804127047A84800B5C16821F03A
:10251000405141F00051C160C16C41F04051C16473
:10252000A3491A200860091D0A6830EA0202FBD19B
:102530004FF0E0214FF08070C1F880029D4B2022C7
:1025400083F80024C1F80001FFF7C2FF00205DF806
:1025500004EBAFE7704710B500B101204FF4807471
:1025600044EA00419448FFF76EFF8B480321C0F80E
:10257000441200BFD0F80012C905FBD5C0F80842CC
:1025800010BD10B502468078FFF74AFF8249D1F8A6
:102590004432012484402343C1F84432C1F8480244
:1025A0009088C1F84C0200BFD1F80002C005FBD5ED
:1025B0004FF48070C1F8080210BD704700B5FFF7F6
:1025C0002FFF7E495DF804EB41EA004089133AE7AA
:1025D00000B5FFF725FF79495DF804EB41EA0040BB
:1025E000774930E700B5FFF71BFF74495DF804EB4E
:1025F00041EA0040891326E700B5FFF711FF6F4954
:102600005DF804EB41EA00406E491CE700B5FFF7B6
:1026100007FF6A495DF804EB41EA0040891312E7BD
:1026200000F00F02012370B503EB82035A4AC2F88F
:10263000283200BFD2F820321C05FBD5C3F30903B2
:102640000024DD1C05E000BFD2F8186241F8046BDD
:10265000641CB4EB950FF7D30021C2F8281241F2A5
:102660004821C140C9070AD1FFF7DAFE4FF4A06143
:1026700041EA0040FFF7DBFE5348FFF7D8FE18465B
:1026800070BD70B513460546434C00F00F000222A2
:1026900002EB8000C4F82802C4F824320020DA1CBF
:1026A00005E000BF51F8046BC4F81C62401CB0EB9D
:1026B000920FF7D30020C4F828022846FFF7B0FE97
:1026C0004FF4A06141EA0040FFF7B1FE3F48FFF739
:1026D000AEFE184670BD2DE9F0412F4DD5F8003201
:1026E000C5F80832180721D52C48FFF7A0FE384856
:1026F000FFF7BDFEC10605D5FFF7EAFEBDE8F041D4
:10270000FDF7D9BD810705D5BDE8F04100F0010016
:10271000FDF7CBBD010709D5400703D5BDE8F04162
:10272000FDF7D0BDBDE8F041FDF7D3BD294E5807F8
:102730004FF001071CD4BDE8F0810024D5F8302209
:1027400007FA04F10A4210D06008C5F8381200BF39
:10275000D5F800128906FBD5D5F81412E2070CD083
:1027600056F8201009B103208847641C202CE5D3BB
:10277000D5F830020028E0D1DDE73CB9490705D59E
:10278000316819B1012088470124D7E756F8201095
:102790000029EAD00220E7E700C000500005FE0053
:1027A00000C00920000180000005D00000C00240E8
:1027B000F4CF005018E000E00005D800000540000C
:1027C00000012000000101000005F2000005FA00F0
:1027D0000002FE00B45600002DE9F047F74E804697
:1027E0004FF080773068BC11F54DB84249D100BF39
:1027F00000BF00BF00BF00BF00BF00BF00BF00BFE1
:1028000000BF00BF00BF00BF00BF00BF00BF00BFD0
:1028100000BF00BF00BF00BF00BF00BF00BF00BFC0
:1028200000BF00BF00BF00BF00BF00BF00BFEC6320
:102830001520FDF779FD0020FDF776FD00F0FF097A
:10284000AC6300BF00BF00BF00BF00BF00BF00BF40
:1028500000BF00BF00BF00BF00BF00BF00BF00BF80
:1028600000BF00BF00BF00BF00BF00BF00BF00BF70
:1028700000BF00BF00BF00BF00BF00BF00BF00BF60
:1028800000BF00BF00BF00BF00BF00BF00BF00BF50
:1028900000BF00BF00BF00BF00BF00BF00BF00BF40
:1028A00000BF00BF00BF00BF00BF00BF00BF00BF30
:1028B00000BF00BF00BF00BF00BF00BF00BF00BF20
:1028C00000BFEC630620FDF72FFDAC6300BF00BF27
:1028D00000BF00BF00BF00BF00BF00BF00BF00BF00
:1028E00000BF00BF00BF00BF00BF00BF00BF00BFF0
:1028F00000BF00BF00BF00BF00BF00BF00BF00BFE0
:1029000000BF00BF00BF00BF00BF00BF00BF00BFCF
:1029100000BF00BF00BF00BF00BF00BF00BF00BFBF
:1029200000BF00BF00BF00BF00BF00BF00BF00BFAF
:1029300000BF00BF00BF00BF00BF00BF00BF00BF9F
:1029400000BF00BF00BF00BF00BF00BFEC6301209D
:10295000FDF7EAFC4FEA8800FDF7E6FC3068B84274
:1029600002D14846FDF7E0FCAC6300BF00BF00BFEA
:1029700000BF00BF00BF00BF00BF00BF00BF00BF5F
:1029800000BF00BF00BF00BF00BF00BF00BF00BF4F
:1029900000BF00BF00BF00BF00BF00BF00BF00BF3F
:1029A00000BF00BF00BF00BF00BFBDE8F0872DE93A
:1029B000FC5F8846044601A9824800F05DFB824D19
:1029C000824E834FF0BB03208DF8000020098DF864
:1029D000010020018DF802004FF000098DF80390EE
:1029E00000BF00BF00BF00BF00BF00BF00BF00BFEF
:1029F00000BF00BF00BF00BF00BF00BF00BF00BFDF
:102A000000BF00BF00BF00BF00BF00BF00BF00BFCE
:102A100000BF00BF00BF00BF00BF00BF00BF00BFBE
:102A2000DFF89CB14FF4802ACBF83CA00421684623
:102A3000FDF781FC00240020FDF776FCC0B28DF884
:102A4000040000E003E018F80410884208D0822057
:102A5000286022203060784638608220BDE8FC9FE4
:102A6000641CB4F5805FE6D3CBF838A000BF00BF8C
:102A700000BF00BF00BF00BF00BF00BF00BF00BF5E
:102A800000BF00BF00BF00BF00BF00BF00BF00BF4E
:102A900000BF00BF00BF00BF00BF00BF00BF00BF3E
:102AA00000BF00BF00BF00BF00BF00BFC5F800905F
:102AB0007846C6F8009038600020CFE72DE9F0474F
:102AC0004FF0000900BF00BF00BF00BF00BF00BF44
:102AD00000BF00BF00BF00BF00BF00BF00BF00BFFE
:102AE00000BF00BF00BF00BF00BF00BF00BF00BFEE
:102AF00000BF00BF00BF00BF00BF00BF00BF00BFDE
:102B000000BF00BF2E4E4FF48025F5639F20FDF7D8
:102B10000BFC0020FDF708FC00F0FF080020FDF78B
:102B200003FCC4B20020FDF7FFFBC1B2B56300BFD8
:102B300000BF00BF00BF00BF00BF00BF00BF00BF9D
:102B400000BF00BF00BF00BF00BF00BF00BF00BF8D
:102B500000BF00BF00BF00BF00BF00BF00BF00BF7D
:102B600000BF00BF00BF00BF00BF00BF00BF164DC9
:102B7000164E174FB8F1C20F01D1202C07D082207A
:102B80002860212030607846386082200DE70B48AD
:102B900014291FD0152920D0162922D0182923D076
:102BA000C0F800900020FFF717FEC5F800907846A7
:102BB000C6F8009038600020F7E600001001001011
:102BC00000C00920A08601006C00001070000010F9
:102BD000740000104FF4801101E04FF40011016007
:102BE000E0E74FF48001FAE74FF08071F7E72DE955
:102BF000F34FC3B0804600244FF0820AFE4DFF4ED3
:102C0000FF4F4FF0210BA14641A9FE4800F034FAD6
:102C100000286CD100F09CFA02208DF800004FEAE9
:102C200018108DF8010004EB08108DF8020044988C
:102C30008DF8039000EB04214FF4807201A801F09D
:102C4000FFFF00BF00BF00BF00BF00BF00BF00BF4D
:102C500000BF00BF00BF00BF00BF00BF00BF00BF7C
:102C600000BF00BF00BF00BF00BF00BF00BF00BF6C
:102C700000BF00BF00BF00BF00BF00BF00BF00BF5C
:102C800000BFE1494FF48020C8634FF48271684669
:102C9000FDF751FBDC494FF48020886300BF00BF83
:102CA00000BF00BF00BF00BF00BF00BF00BF00BF2C
:102CB00000BF00BF00BF00BF00BF00BF00BF00BF1C
:102CC00000BF00BF00BF00BF00BF00BF00BF00BF0C
:102CD00000BF00BF00BF00BF00BF00BF641CE4B264
:102CE000102C91D341A9C74800F0C6F948B1C5F8E6
:102CF00000A07846C6F800B03860822045B0BDE834
:102D0000F08F00F06FFAC5F800907846C6F8009092
:102D100038600020F2E72DE9F04F89B0DFF8D88263
:102D20005FEA020B4FF0000607910FD04FF4805579
:102D300001462A46684601F079FFDDE9004728464A
:102D4000FDF714FB5FEA00090CD016E08621AB48C2
:102D5000C8F80010092101607946A9480160862061
:102D600009B0CCE78221A548C8F8001022210160F3
:102D70007946A34801608220F2E7ABEB0605C7F570
:102D800080504FF0000AA84200D20546B5F5805F9A
:102D900004D02046494600F0A3FCD8B907982A463B
:102DA000811907EB090001F04BFF204600F01DFCE4
:102DB00080B920464946FFF71AFF58B920464946D0
:102DC000FFF7F5FD78B10AF1010000F0FF0ABAF152
:102DD000030F05D3484601F069FED8F80000BFE7AD
:102DE000BAF1000FE1D12E440027641C5E45C4D324
:102DF000484601F05BFE81490020C8F800000860E9
:102E000079467F4801600020AAE72DE9FF4F8DB089
:102E10000D46DDF868900026774C07935FEA0901BC
:102E20003FD04FF4805701463A46684601F0FEFE17
:102E3000DDE900B10C913A46691C684601F0F6FEE6
:102E4000DDE90010CDE904013A4668460F9901F02A
:102E5000EDFEDDE9008500BFA9EB0607C5F5805052
:102E6000B84200D2074625B1D8457CD10C9885429E
:102E700079D14FF48050FDF779FA5FEA000A1BD050
:102E8000D8454FD10C9885424CD12A464FEA08309C
:102E9000514600F0FEFA000618D5504601F006FE35
:102EA00079E0862020605548092101607846544920
:102EB0000860862011B022E7822020604F4822213E
:102EC000016079464E4801608220F3E7059880450D
:102ED00009D1049901EB0030C1F58052514400F052
:102EE000D8FA0006D9D4404600F07FFB0006D4D4BF
:102EF00007983A46811905EB0A0001F0A1FEEA198C
:102F00004FEA0830514601F0DCF90006C5D40599B6
:102F1000884533D1049800EB01300499C1F5805203
:102F2000514427E0059988450AD1049800EB013007
:102F30000499C1F58052514600F0ABFA0006ACD4BA
:102F4000404600F052FB0006A7D407983A46811984
:102F50000F98304401F0B5F900069ED405998845D4
:102F60000CD1049800E00DE000EB01300499C1F5AC
:102F70008052514601F0A5F900068ED4504601F06A
:102F800095FD0AE007983A4681190F98304401F000
:102F900098F9000601D520688CE73E44002508F129
:102FA00001084E45FFF458AF144900202060086026
:102FB00078461349086000207CE714480068704791
:102FC0004FF4805070472DE9F04FDFF82C80DFF888
:102FD0002CB089B00F0004464FF0000633D04FF4F8
:102FE000805501462A46684601F020FEDDE900A131
:102FF00005912A4621460BE06C000010700000107D
:1030000074000010A086010000C00920100100100B
:1030100006A801F00BFEDDE906404FF00009BD1BDC
:10302000C0F58051A94200D20D4620B1544515D1BA
:103030000599884212D1204600F0D7FA00060DD536
:10304000D8F800008CE68621C8F800100921CBF8DA
:10305000001079463B480160862081E62E44641CBE
:103060004846BE42DBD3C8F800007946CBF80000E2
:1030700034480160002073E62DE9F041324C0F46E0
:103080000646A56806E0A068401BB04202D30120B6
:10309000BDE8F081384600F003F80028F3D1F7E7E7
:1030A00070B5044600BF00BF00BF00BF00BF00BF37
:1030B00000BF00BF00BF00BF00BF00BF00BF00BF18
:1030C00000BF00BF00BF00BF00BF00BF00BF00BF08
:1030D00000BF00BF00BF00BF00BF00BF00BF00BFF8
:1030E00000BF00BF194E4FF48025F5630520FDF7A2
:1030F0001BF90020FDF718F92070B56300BF00BF71
:1031000000BF00BF00BF00BF00BF00BF00BF00BFC7
:1031100000BF00BF00BF00BF00BF00BF00BF00BFB7
:1031200000BF00BF00BF00BF00BF00BF00BF00BFA7
:1031300000BF00BF00BF00BF00BF00BF207800F08D
:10314000010070BD740000100000094000C009209B
:1031500070B500BF00BF00BF00BF00BF00BF00BF11
:1031600000BF00BF00BF00BF00BF00BF00BF00BF67
:1031700000BF00BF00BF00BF00BF00BF00BF00BF57
:1031800000BF00BF00BF00BF00BF00BF00BF00BF47
:1031900000BFFE4C4FF48025E5630620FDF7C4F820
:1031A000A56300BF00BF00BF00BF00BF00BF00BFDE
:1031B00000BF00BF00BF00BF00BF00BF00BF00BF17
:1031C00000BF00BF00BF00BF00BF00BF00BF00BF07
:1031D00000BF00BF00BF00BF00BF00BF00BF00BFF7
:1031E00000BF70BD70B500BF00BF00BF00BF00BF13
:1031F00000BF00BF00BF00BF00BF00BF00BF00BFD7
:1032000000BF00BF00BF00BF00BF00BF00BF00BFC6
:1032100000BF00BF00BF00BF00BF00BF00BF00BFB6
:1032200000BF00BF00BFD94C4FF48025E5630420E8
:10323000FDF77AF8A56300BF00BF00BF00BF00BF65
:1032400000BF00BF00BF00BF00BF00BF00BF00BF86
:1032500000BF00BF00BF00BF00BF00BF00BF00BF76
:1032600000BF00BF00BF00BF00BF00BF00BF00BF66
:1032700000BF00BF00BF70BD70B5064600BF00BFF5
:1032800000BF00BF00BF00BF00BF00BF00BF00BF46
:1032900000BF00BF00BF00BF00BF00BF00BF00BF36
:1032A00000BF00BF00BF00BF00BF00BF00BF00BF26
:1032B00000BF00BF00BF00BF00BF00BFB34D4FF451
:1032C0008024EC635020FDF72FF8AC6300BF00BFF3
:1032D00000BF00BF00BF00BF00BF00BF00BF00BFF6
:1032E00000BF00BF00BF00BF00BF00BF00BF00BFE6
:1032F00000BF00BF00BF00BF00BF00BF00BF00BFD6
:1033000000BF00BF00BF00BF00BF00BF00BF00BFC5
:1033100000BF00BF00BF00BF00BF00BF00BF00BFB5
:1033200000BF00BF00BF00BF00BF00BF00BF00BFA5
:1033300000BF00BF00BF00BF00BF00BF00BF00BF95
:1033400000BF00BF00BF00BF00BF00BFEC63012093
:10335000FCF7EAFFB000FCF7E7FFAC6300BF00BF7B
:1033600000BF00BF00BF00BF00BF00BF00BF00BF65
:1033700000BF00BF00BF00BF00BF00BF00BF00BF55
:1033800000BF00BF00BF00BF00BF00BF00BF00BF45
:1033900000BF00BF00BF00BF00BF00BF70BD2DE970
:1033A000FE430F46044602A9794800F0BCFD794D62
:1033B000794EDFF8E88148B18220286022207946E2
:1033C00030608220C8F80010BDE8FE839DF8080038
:1033D000800701D4FFF7BCFE02208DF80000200C0E
:1033E0008DF80100200A8DF802008DF803408DF859
:1033F000047000BF00BF00BF00BF00BF00BF00BF20
:1034000000BF00BF00BF00BF00BF00BF00BF00BFC4
:1034100000BF00BF00BF00BF00BF00BF00BF00BFB4
:1034200000BF00BF00BF00BF00BF00BF00BF00BFA4
:1034300000BF564F4FF48024FC6305216846FCF71B
:103440007AFFBC6300BF00BF00BF00BF00BF00BF6A
:1034500000BF00BF00BF00BF00BF00BF00BF00BF74
:1034600000BF00BF00BF00BF00BF00BF00BF00BF64
:1034700000BF00BF00BF00BF00BF00BF00BF00BF54
:1034800000BF00BF0020286079463060C8F80010F7
:103490009AE72DE9FC5F3F4D3F4E404F5FEA020A3D
:1034A0008B4604464FF000080DD001A9384800F0C3
:1034B0003AFD80B182202860212030607846386053
:1034C0008220BDE8FC9FC5F800807846C6F80080E1
:1034D00038600020F5E703208DF80000200C8DF8FF
:1034E0000100200A8DF802008DF8034000BF00BFE4
:1034F00000BF00BF00BF00BF00BF00BF00BF00BFD4
:1035000000BF00BF00BF00BF00BF00BF00BF00BFC3
:1035100000BF00BF00BF00BF00BF00BF00BF00BFB3
:1035200000BF00BF00BF00BF00BF00BF174C4FF47B
:103530008029C4F83C9004216846FCF7FCFE514603
:103540005846FCF704FFC4F8389000BF00BF00BF26
:1035500000BF00BF00BF00BF00BF00BF00BF00BF73
:1035600000BF00BF00BF00BF00BF00BF00BF00BF63
:1035700000BF00BF00BF00BF00BF00BF00BF00BF53
:1035800000BF00BF00BF00BF00BF9CE700C0092014
:10359000A08601006C000010700000107400001084
:1035A0002DE9F05FFF4EDFF80094DFF800A415006E
:1035B00083460F464FF000080ED000240AE0395D24
:1035C0000BEB0400FFF7EBFE000602D53068BDE808
:1035D000F09F641CAC42F2D3C6F800807946C9F86B
:1035E00000800020CAF80010F1E72DE9FC470446EE
:1035F00001A9EF4800F097FCEA4DEB4EDFF8AC93E1
:1036000048B1822028602220794630608220C9F8A3
:103610000010BDE8FC879DF80400800701D4FFF787
:1036200097FD20208DF8000020098DF80100200171
:103630008DF8020000248DF8034000BF00BF00BFDA
:1036400000BF00BF00BF00BF00BF00BF00BF00BF82
:1036500000BF00BF00BF00BF00BF00BF00BF00BF72
:1036600000BF00BF00BF00BF00BF00BF00BF00BF62
:1036700000BF00BF00BF00BF00BFDFF838834FF4BA
:103680008027C8F83C7004216846FCF754FEC8F84F
:10369000387000BF00BF00BF00BF00BF00BF00BF49
:1036A00000BF00BF00BF00BF00BF00BF00BF00BF22
:1036B00000BF00BF00BF00BF00BF00BF00BF00BF12
:1036C00000BF00BF00BF00BF00BF00BF00BF00BF02
:1036D00000BF2C60794634600020C9F8001098E7DC
:1036E0002DE9FC478A46044601A9B14800F01BFCBD
:1036F000AC4DAD4EDFF8B49240B18220286022205C
:10370000794630608220C9F8001082E703208DF8E6
:10371000000020098DF8010020018DF8020000242E
:103720008DF8034000BF00BF00BF00BF00BF00BF57
:1037300000BF00BF00BF00BF00BF00BF00BF00BF91
:1037400000BF00BF00BF00BF00BF00BF00BF00BF81
:1037500000BF00BF00BF00BF00BF00BF00BF00BF71
:1037600000BF00BFDFF84C824FF48027C8F83C70E0
:1037700004216846FCF7DFFDB9115046FCF7E7FD70
:10378000C8F8387000BF00BF00BF00BF00BF00BF57
:1037900000BF00BF00BF00BF00BF00BF00BF00BF31
:1037A00000BF00BF00BF00BF00BF00BF00BF00BF21
:1037B00000BF00BF00BF00BF00BF00BF00BF00BF11
:1037C00000BF00BF2C60794634600020C9F80010AB
:1037D0001FE72DE9F34F83B0044601A9744800F0B8
:1037E000A2FB704D704E714F4FF0820818B121202E
:1037F000C5F800806CE09DF80400800701D4FFF755
:10380000A7FCAD208DF8000020098DF801002001F3
:103810008DF802004FF0000B8DF803B000BF00BF21
:1038200000BF00BF00BF00BF00BF00BF00BF00BFA0
:1038300000BF00BF00BF00BF00BF00BF00BF00BF90
:1038400000BF00BF00BF00BF00BF00BF00BF00BF80
:1038500000BF00BF00BF00BF00BF00BFDFF8549132
:103860004FF4802A5446C9F83CA004216846FCF76E
:1038700062FD02210498FCF75EFDC9F8384000BFE4
:1038800000BF00BF00BF00BF00BF00BF00BF00BF40
:1038900000BF00BF00BF00BF00BF00BF00BF00BF30
:1038A00000BF00BF00BF00BF00BF00BF00BF00BF20
:1038B00000BF00BF00BF00BF00BF00BF00BF0224A9
:1038C00001A93B4800F02FFB48B12220C5F8008039
:1038D000306078463860822005B0BDE8F08F00BFC8
:1038E00000BF00BF00BF00BF00BF00BF00BF00BFE0
:1038F00000BF00BF00BF00BF00BF00BF00BF00BFD0
:1039000000BF00BF00BF00BF00BF00BF00BF00BFBF
:1039100000BF00BF00BF00BF00BF00BF00BFC9F8AD
:103920003CA0AD20FCF700FD049802212044FCF7E8
:1039300002FDC9F838A000BF00BF00BF00BF00BF34
:1039400000BF00BF00BF00BF00BF00BF00BF00BF7F
:1039500000BF00BF00BF00BF00BF00BF00BF00BF6F
:1039600000BF00BF00BF00BF00BF00BF00BF00BF5F
:1039700000BF00BF00BFA41CA4B2B4F5805F9FD3FA
:1039800001A90B4800F0CFFA00287FF430AFFFF711
:1039900029FCC5F800B07846C6F800B038600020B1
:1039A0009AE700006C000010700000107400001016
:1039B000A086010000C0092070B5FD4DFD4EFE4CF3
:1039C0002AB1FFF766FD000609D5206870BD862084
:1039D00020600920286078463060862070BD002075
:1039E0002060286078463060002070BD2DE9F04FDF
:1039F00089B0DFF8C483DFF8B8B35FEA02094FF09B
:103A0000000607910FD04FF4805501462A466846BC
:103A100001F00CF9DDE900472846FCF7A7FC5FEA56
:103A2000000A0CD016E08621C8F800100921CBF856
:103A300000107946DF480160862009B04DE78221F9
:103A4000C8F800102221CBF800107946D94801604F
:103A50008220F2E7A9EB0605C7F58050A84200D204
:103A60000546B5F5805F04D020465146FFF738FE85
:103A700080B92046FFF7B9FD60B907982A46811939
:103A800007EB0A0001F0DCF82E4420465146FFF710
:103A9000A0FE28B1504601F009F8D8F80000CCE7A4
:103AA0000027641C4E45D5D3504600F0FFFF002090
:103AB000C8F800007946CBF80000BE48016000203D
:103AC000BBE72DE9FF4F8DB00D46DDF8689000266D
:103AD000B94C07935FEA09013FD04FF48057014684
:103AE0003A46684601F0A2F8DDE900B10C913A4689
:103AF000691C684601F09AF8DDE90010CDE904017F
:103B00003A4668460F9901F091F8DDE9008500BF5B
:103B1000A9EB0607C5F58050B84200D2074625B18B
:103B2000D8457CD10C98854279D14FF48050FCF770
:103B30001DFC5FEA000A1BD0D8454FD10C98854286
:103B40004CD12A464FEA08305146FFF7A2FC000646
:103B500018D5504600F0AAFF79E0862020609448EE
:103B600009210160784693490860862011B0B4E6C7
:103B7000822020608E482221016079468D480160B4
:103B80008220F3E70598804509D1049901EB0030C4
:103B9000C1F580525144FFF77CFC0006D9D4404661
:103BA000FFF723FD0006D4D407983A46811905EBA8
:103BB0000A0001F045F8EA194FEA08305146FFF7CC
:103BC000EFFC0006C5D40599884533D1049800EB75
:103BD00001300499C1F58052514427E00599884588
:103BE0000AD1049800EB01300499C1F58052514686
:103BF000FFF74FFC0006ACD44046FFF7F6FC00068A
:103C0000A7D407983A4681190F983044FFF7C8FCAB
:103C100000069ED4059988450CD1049800E00DE07B
:103C200000EB01300499C1F580525146FFF7B8FC12
:103C300000068ED4504600F039FF0AE007983A4655
:103C400081190F983044FFF7ABFC000601D52068BE
:103C50008CE73E44002508F101084E45FFF458AFBB
:103C600053490020206008607846524908600020CF
:103C70007CE72DE9F0474FF0000900BF00BF00BF0F
:103C800000BF00BF00BF00BF00BF00BF00BF00BF3C
:103C900000BF00BF00BF00BF00BF00BF00BF00BF2C
:103CA00000BF00BF00BF00BF00BF00BF00BF00BF1C
:103CB00000BF00BF00BF00BF00BF404E4FF48025D3
:103CC000F5639F20FCF730FB0020FCF72DFB00F094
:103CD000FF080020FCF728FBC4B20020FCF724FBFF
:103CE000C1B2B56300BF00BF00BF00BF00BF00BFCF
:103CF00000BF00BF00BF00BF00BF00BF00BF00BFCC
:103D000000BF00BF00BF00BF00BF00BF00BF00BFBB
:103D100000BF00BF00BF00BF00BF00BF00BF00BFAB
:103D200000BF00BF244D224E224FB8F1BF0F03D178
:103D3000252C0AD0262C08D0822028602120306033
:103D4000784638608220BDE8F0871D48412912D0AE
:103D50004FF48002422912D04A2910D0C0F80090B6
:103D60000020FFF789FAC5F800907846C6F8009061
:103D700038600020E7E74FF400110160F0E70260CF
:103D8000EEE72DE9F84F69460E4800F0CCF882279F
:103D9000094C074D074E4FF0220A002862D19DF8CA
:103DA0000000800701D4FFF7D3F900BF00BF0BE08C
:103DB00070000010740000106C00001000C009209A
:103DC00014010010A086010000BF00BF00BF00BFAB
:103DD00000BF00BF00BF00BF00BF00BF00BF00BFEB
:103DE00000BF00BF00BF00BF00BF00BF00BF00BFDB
:103DF00000BF00BF00BF00BF00BF00BF00BF00BFCB
:103E000000BF00BFDFF8EC914FF48028C9F83C8078
:103E10006020FCF789FAC9F8388000BF00BF00BFF6
:103E200000BF00BF00BF00BF00BF00BF00BF00BF9A
:103E300000BF00BF00BF00BF00BF00BF00BF00BF8A
:103E400000BF00BF00BF00BF00BF00BF00BF00BF7A
:103E500000BF00BF00BF00BF00BF6946664800F05A
:103E600062F838B127607846C5F800A0306082203B
:103E7000BDE8F88F00202060286078463060002080
:103E8000F6E75E48006870474FF4805070472DE9B0
:103E9000F04FDFF86C81DFF86CB189B00F00044699
:103EA0004FF0000626D04FF4805501462A4668465A
:103EB00000F0BCFEDDE900A105912A46214606A8D6
:103EC00000F0B4FEDDE906404FF00009BD1BC0F56F
:103ED0008051A94200D20D4620B1544515D1059913
:103EE000884212D12046FFF780FB00060DD5D8F896
:103EF0000000A2E58621C8F800100921CBF80010C7
:103F0000794641480160862097E52E44641C484666
:103F1000BE42DBD3C8F800007946CBF800003A482F
:103F20000160002089E52DE9F041384C0F46064636
:103F3000A56806E0A068401BB04202D30120BDE89E
:103F4000F081384600F003F80028F3D1F7E770B5A8
:103F5000044600BF00BF00BF00BF00BF00BF00BFDE
:103F600000BF00BF00BF00BF00BF00BF00BF00BF59
:103F700000BF00BF00BF00BF00BF00BF00BF00BF49
:103F800000BF00BF00BF00BF00BF00BF00BF00BF39
:103F900000BF184E4FF48025F5630520FCF7C4F9E7
:103FA0000020FCF7C1F92070B56300BF00BF00BF5F
:103FB00000BF00BF00BF00BF00BF00BF00BF00BF09
:103FC00000BF00BF00BF00BF00BF00BF00BF00BFF9
:103FD00000BF00BF00BF00BF00BF00BF00BF00BFE9
:103FE00000BF00BF00BF00BF00BF207800F001008D
:103FF00070BD000000C0092020A1070014010010BE
:104000006C000010700000107400001000000940E7
:104010002DE9FF4703A9FE4800F063FBFD4DFE4E6E
:10402000DFF8F89350B18220286021207946306073
:104030008220C9F8001004B0BDE8F0879DF80C009C
:10404000800701D4FFF784F842208DF80000002497
:10405000CDF80140CDF80540ADF8094000BF00BFE4
:1040600000BF00BF00BF00BF00BF00BF00BF00BF58
:1040700000BF00BF00BF00BF00BF00BF00BF00BF48
:1040800000BF00BF00BF00BF00BF00BF00BF00BF38
:1040900000BF00BF00BF00BF00BF00BFDFF88083CC
:1040A0004FF48027C8F83C700B216846FCF743F9B1
:1040B000C8F8387000BF00BF00BF00BF00BF00BF1E
:1040C00000BF00BF00BF00BF00BF00BF00BF00BFF8
:1040D00000BF00BF00BF00BF00BF00BF00BF00BFE8
:1040E00000BF00BF00BF00BF00BF00BF00BF00BFD8
:1040F00000BF00BF2C60794634600020C9F8001072
:1041000099E72DE9F34F85B0044603A9C04800F0B4
:10411000E8FAC04DC04EC14F4FF0820B18B12120BC
:10412000C5F800B060E0FFF713F842208DF80000FA
:104130004FF0000ACDF801A0CDF805A0ADF809A018
:1041400000BF00BF00BF00BF00BF00BF00BF00BF77
:1041500000BF00BF00BF00BF00BF00BF00BF00BF67
:1041600000BF00BF00BF00BF00BF00BF00BF00BF57
:1041700000BF00BF00BF00BF00BF00BF00BF00BF47
:10418000DFF89C924FF48028C9F83C800B216846E8
:10419000FCF7D1F8C9F8388000BF00BF00BF00BFEE
:1041A00000BF00BF00BF00BF00BF00BF00BF00BF17
:1041B00000BF00BF00BF00BF00BF00BF00BF00BF07
:1041C00000BF00BF00BF00BF00BF00BF00BF00BFF7
:1041D00000BF00BF00BF00BF03A98D4800F081FAF7
:1041E00048B12220C5F800B030607846386082209F
:1041F00007B0BDE8F08F9DF80C00800701D4FEF7F2
:10420000A7FF02208DF80000200C8DF80100200A85
:104210008DF8020006988DF803408DF8040000BF69
:1042200000BF00BF00BF00BF00BF00BF00BF00BF96
:1042300000BF00BF00BF00BF00BF00BF00BF00BF86
:1042400000BF00BF00BF00BF00BF00BF00BF00BF76
:1042500000BF00BF00BF00BF00BF00BF00BF44469B
:10426000C846C9F83C4005216846FCF764F8C8F820
:10427000384000BF00BF00BF00BF00BF00BF00BF8D
:1042800000BF00BF00BF00BF00BF00BF00BF00BF36
:1042900000BF00BF00BF00BF00BF00BF00BF00BF26
:1042A00000BF00BF00BF00BF00BF00BF00BF00BF16
:1042B00000BFC5F800A07846C6F800A0386000200E
:1042C00096E72DE9F05F534EDFF84C91DFF84CA1F3
:1042D000150083460F464FF000080ED000240AE078
:1042E000395D0BEB0400FFF70CFF000602D53068C8
:1042F000BDE8F09F641CAC42F2D3C6F8008079465A
:10430000C9F800800020CAF80010F1E72DE9F34F4A
:104310000024404D404E414FC3B080464FF0820ACA
:104320004FF0210BA14641A9394800F0DAF90028E5
:104330007CD19DF80401800701D4FEF709FF02201B
:104340008DF800004FEA18108DF8010004EB0810FA
:104350008DF8020044988DF8039000EB04214FF48F
:10436000807201A800F06CFC00BF00BF00BF00BF5E
:1043700000BF00BF00BF00BF00BF00BF00BF00BF45
:1043800000BF00BF00BF00BF00BF00BF00BF00BF35
:1043900000BF00BF00BF00BF00BF00BF00BF00BF25
:1043A00000BF00BF00BF00BF1D494FF48020C8639D
:1043B0004FF482716846FBF7BEFF19494FF4802025
:1043C000886300BF00BF00BF00BF00BF00BF00BFC9
:1043D00000BF00BF00BF00BF00BF00BF00BF00BFE5
:1043E00000BF00BF00BF00BF00BF00BF00BF00BFD5
:1043F00000BF00BF00BF00BF00BF00BF00BF00BFC5
:1044000000BF641CE4B2102C8DD341A900480AE01F
:10441000A08601006C0000107000001074000010F5
:1044200000C0092002E000F05CF940B1C5F800A02E
:104430007846C6F800B03860822045B0D9E6FEF76D
:10444000D1FEC5F800907846C6F80090386000208C
:10445000F3E72DE9F04F89B0DFF85483DFF854B368
:104460005FEA02094FF0000607910FD04FF4805524
:1044700001462A46684600F0D9FBDDE90047284698
:10448000FBF774FF5FEA000A0CD016E08621C8F83B
:1044900000100921CBF800107946C748016086203A
:1044A00009B0A6E68221C8F800102221CBF800103E
:1044B0007946C14801608220F2E7A9EB0605C7F5FD
:1044C0008050A84200D20546B5F5805F04D0204652
:1044D0005146FFF705F980B92046FFF786F860B925
:1044E00007982A46811907EB0A0000F0A9FB2E4421
:1044F00020465146FFF70AFF28B1504600F0D6FA91
:10450000D8F80000CCE70027641C4E45D5D35046B0
:1045100000F0CCFA0020C8F800007946CBF8000083
:10452000A54801600020BBE72DE9FF4F8DB00D4687
:10453000DDF8689000269E4C07935FEA09013ED0A3
:104540004FF4805701463A46684600F06FFBDDE9BC
:1045500000B10C913A46691C684600F067FBDDE942
:104560000010CDE904013A4668460F9900F05EFB61
:10457000DDE90085A9EB0607C5F58050B84200D2F9
:10458000074625B1D8457CD10C98854279D14FF4A6
:104590008050FBF7EBFE5FEA000A1BD0D8454FD1F5
:1045A0000C9885424CD12A464FEA08305146FEF716
:1045B00070FF000618D5504600F078FA79E08620A2
:1045C00020607C480921016078467B49086086208C
:1045D00011B00EE6822020607648222101607946E3
:1045E000754801608220F3E70598804509D1049958
:1045F00001EB0030C1F580525144FEF74AFF00063E
:10460000D9D44046FEF7F1FF0006D4D407983A46C5
:10461000811905EB0A0000F013FBEA194FEA083094
:104620005146FFF74EFE0006C5D40599884533D1A3
:10463000049800EB01300499C1F58052514427E001
:10464000059988450AD1049800EB01300499C1F519
:1046500080525146FEF71DFF0006ACD44046FEF7DF
:10466000C4FF0006A7D407983A4681190F98304432
:10467000FFF727FE00069ED4059988450CD10498C3
:1046800000E00DE000EB01300499C1F58052514685
:10469000FFF717FE00068ED4504600F007FA0AE036
:1046A00007983A4681190F983044FFF70AFE000632
:1046B00001D520688CE73E44002508F101084E45ED
:1046C000FFF458AF3B4900202060086078463A4923
:1046D000086000207CE74FF4800070474FF4805062
:1046E00070472DE9F041354C0F460646A56806E0B7
:1046F000A068401BB04202D30120BDE8F0813846DB
:1047000000F003F80028F3D1F7E770B5044600BFC6
:1047100000BF00BF00BF00BF00BF00BF00BF00BFA1
:1047200000BF00BF00BF00BF00BF00BF00BF00BF91
:1047300000BF00BF00BF00BF00BF00BF00BF00BF81
:1047400000BF00BF00BF00BF00BF00BF00BF1C4EC6
:104750004FF48025F5630520FBF7E6FD0020FBF70D
:10476000E3FD2070B56300BF00BF00BF00BF00BF06
:1047700000BF00BF00BF00BF00BF00BF00BF00BF41
:1047800000BF00BF00BF00BF00BF00BF00BF00BF31
:1047900000BF00BF00BF00BF00BF00BF00BF00BF21
:1047A00000BF00BF00BF207800F0010070BD000016
:1047B0006C00001070000010740000100000094030
:1047C00000C0092000207047AE4982200860AE4931
:1047D000212008607846AD49086082207047A949C9
:1047E00082200860A849222008607846A74908600E
:1047F00082207047A34982200860A34922200860D4
:104800007846A24908608220704770B5002400BF36
:1048100000BF00BF00BF00BF00BF00BF00BF00BFA0
:1048200000BF00BF00BF00BF00BF00BF00BF00BF90
:1048300000BF00BF00BF00BF00BF00BF00BF00BF80
:1048400000BF00BF00BF00BF00BF00BF00BF904E51
:104850004FF48025F5639F20FBF766FD0020FBF7F2
:1048600063FD60F307040020FBF75EFD60F30F2497
:104870000020FBF759FD60F31744B56300BF00BF8C
:1048800000BF00BF00BF00BF00BF00BF00BF00BF30
:1048900000BF00BF00BF00BF00BF00BF00BF00BF20
:1048A00000BF00BF00BF00BF00BF00BF00BF00BF10
:1048B00000BF00BF00BF00BF00BF00BF7549601A46
:1048C0008C421AD00BDCA4F1C204B4F5A11414D0AC
:1048D000B4F5803F11D0B4F5003F0BD10DE06E4927
:1048E000401805D06D49401809D06D49C84201D122
:1048F000022400E00024204670BD0324FBE70424CA
:10490000FFF786FBF7E76748007828B1664900EBB8
:10491000C00051F8200000475A49822008605A49D7
:10492000212008607846594908608220704770B598
:10493000FFF76BFF5B49544D544E524C087050B119
:10494000594900EBC00001EB8000806880470006F9
:1049500009D5206870BD822020602120286078461B
:104960003060822070BD0020206028607846306072
:10497000002070BD2DE9F0414A4B434D434E1B785A
:10498000404C63B19AB1484F03EBC30307EB830379
:104990001B699847000612D52068BDE8F081822087
:1049A000206021202860784630608220F5E786204C
:1049B000206009202860784630608620EDE70020DE
:1049C00020602860784630600020E6E72DE9F0415D
:1049D000344B2D4D2D4E1B782A4C5BB192B1324F8A
:1049E00003EBC30307EB83039B699847000611D5CC
:1049F0002068D2E78220206022202860784630603C
:104A00008220CAE78620206009202860784630602E
:104A10008620C2E7002020602860784630600020B1
:104A2000BBE7F8B51F4C184D184E2778154CDDF82C
:104A300018C087B1BCF1000F15D0CDF800C0DFF869
:104A400068C007EBC7070CEB8707FF69B84700068C
:104A500011D52068F8BD8220206022202860784689
:104A600030608220F8BD86202060092028607846CA
:104A700030608620F8BD00202060286078463060D5
:104A80000020F8BD6C0000107000001074000010D1
:104A900000C00920C220180003FBD6FF00FFFEFF64
:104AA0000001F8FF18010010F456000070B504462C
:104AB000051F00F061F90068002C14BF446870BD48
:104AC000002C18BFAC423CBF20466468F8D3016894
:104AD0000A18AA4218BF456003D12A680546114446
:104AE000016028684119A1421CBF6C6070BD6168FB
:104AF000696021680844286070BD2DE9F0410E46C8
:104B00000446002020622046E168884730B325280B
:104B100005D0D4E901219047206A401CF2E7E16802
:104B2000204600278847050018D0A5F14100192824
:104B300002D820354FF400673246294620462760C8
:104B4000FBF7FEFA40B1012804D0F61D26F0070657
:104B50000836D8E7361DD6E72846DAE7206ABDE8EA
:104B6000F08170B50C460546012A05D028788006EC
:104B700000D5EA69002302E0012305E05B1C9342B3
:104B800002D2E05C0028F9D1A869E618C01AA86131
:104B9000286A184428622846AFF3008004E0D5E96B
:104BA000012114F8010B9047B442F8D32846AFF323
:104BB000008070BD2DE9F04106460024106875297B
:104BC000314616A510D0AFF30080002802DA40422B
:104BD00013A507E031688A0701D512A502E049074D
:104BE00004D511A5012401E0AFF3008000210A22C1
:104BF00006F1240709E0B0FBF2FCB0FBF2F302FB84
:104C00001C00303078541846491C0028F3D1234644
:104C10002A463046BDE8F04100F0FEB80000000032
:104C20002D0000002B0000002000000010B591FBBB
:104C3000F2F491FBF2F302FB1411C0E9003110BD54
:104C4000032A40F2308010F0030C00F0158011F8B8
:104C5000013BBCF1020F624498BF11F801CB00F890
:104C6000013B38BF11F8013BA2F1040298BF00F8E4
:104C700001CB38BF00F8013B11F0030300F02580A1
:104C8000083AC0F0088051F8043B083A51F804CBC8
:104C9000A0E80810F5E7121D5CBF51F8043B40F88E
:104CA000043BAFF30080D20724BF11F8013B11F899
:104CB00001CB48BF11F8012B24BF00F8013B00F8DD
:104CC00001CB48BF00F8012B704710B5203AC0F067
:104CD0000B80B1E81850203AA0E81850B1E81850FD
:104CE000A0E81850BFF4F5AF5FEA027C24BFB1E83A
:104CF0001850A0E8185044BF18C918C0BDE81040AB
:104D00005FEA827C24BF51F8043B40F8043B08BFB3
:104D10007047D20728BF31F8023B48BF11F8012B7A
:104D200028BF20F8023B48BF00F8012B70474FF026
:104D300000020429C0F0128010F0030C00F003817F
:104D4000CCF1040CBCF1020F18BF00F8012BA8BF76
:104D500020F8022BA1EB0C0100F0F5B85FEAC17C52
:104D600024BF00F8012B00F8012B48BF00F8012BED
:104D7000704770477047704700487047601D0010CB
:104D80007047704738B504460A4600206946AFF3BD
:104D90000080002808BF38BD02460099204600F078
:104DA000FBF8012038BD012000F010B9F8B5AFF3D1
:104DB0000080054600200C46102000BF0646A819BA
:104DC000A0420DD9324669460020AFF300800700AB
:104DD00008BF00F0FBF80098A04218BF0546C419B0
:104DE000FFF7CAFF05600746F01D20F007004619CF
:104DF000284600F00AF8B44208BFF8BDA21B3146AD
:104E00003868BDE8F84000F0C7B800210160C0E98B
:104E100001107047102070472DE9F0470D46994664
:104E20009246044600F124080168880604D5E0692A
:104E300021F01001216000E00120A84201DD471BA4
:104E400000E00027A1697A1902EB0900081AA061A5
:104E50002078C00602D42046AFF30080002608E088
:104E6000D4E901211AF806009047206A401C761CFC
:104E700020624E45F4DB2078C0060AD52046AFF309
:104E8000008006E0D4E9012130209047206A401CD0
:104E90002062381EA7F10107F4DC07E0D4E9012104
:104EA00018F805009047206A401C2062281EA5F1D2
:104EB0000105F3DC2046AFF300802078000602D520
:104EC0000220BDE8F0870120FBE7000001694A1CD1
:104ED00002610878704700B58FB0CDE9013100213B
:104EE000059105497944CDE9031011466846FFF75D
:104EF00004FE0FB000BD0000E5FFFFFF0A6802F8E6
:104F0000010B0A607047D1E900239A4202D2531C78
:104F10000B601070704710B5436913B1AFF3008098
:104F200001E0FFF71EFE012010BD127800F1240100
:104F30000A7000224A700122EDE711684FF0FF323B
:104F4000E9E74FF0000200B5134694469646203933
:104F500022BFA0E80C50A0E80C50B1F12001BFF432
:104F6000F7AF090728BFA0E80C5048BF0CC05DF898
:104F700004EB890028BF40F8042B08BF704748BFE6
:104F800020F8022B11F0804F18BF00F8012B70475A
:104F900000487047581D0010034640688C460028A2
:104FA00018BF88423CBF03464068F8D318681844CD
:104FB000884207D00CF1030020F00700001D411AC1
:104FC000521A0146081D0A60FFF770BD10B500F0C7
:104FD00039F8BDE8104000F02FB870477546FFF76C
:104FE000D7FFAE4605006946534620F007008546C8
:104FF00018B020B5FBF7EAF8BDE820404FF00006F6
:105000004FF000074FF000084FF0000B21F00701B0
:10501000AC46ACE8C009ACE8C009ACE8C009ACE8F3
:10502000C0098D46704710B50446AFF30080204696
:10503000BDE81040FBF79DB8002801D000F02AB869
:105040007047000010B5012805D0002103A000F032
:1050500027F8012010BD09A1F8E700005349475285
:10506000544D454D3A204F7574206F662068656138
:1050700070206D656D6F7279000000003A20486500
:105080006170206D656D6F727920636F72727570DB
:105090007465640001491820ABBEFEE726000200DB
:1050A00070B505460C460A2000E06D1C00F011F8B2
:1050B00035B128780028F8D102E0641C00F009F826
:1050C00014B120780028F8D1BDE870400A20AFF371
:1050D000008008B569468DF800000320ABBE08BD0E
:1050E00000050F0A1B1E141133363C39282D2722C8
:1050F00063666C69787D777250555F5A4B4E4441B8
:10510000C3C6CCC9D8DDD7D2F0F5FFFAEBEEE4E1A7
:10511000A0A5AFAABBBEB4B193969C99888D878297
:1051200083868C89989D9792B0B5BFBAABAEA4A187
:10513000E0E5EFEAFBFEF4F1D3D6DCD9C8CDC7C277
:1051400040454F4A5B5E545173767C79686D676267
:1051500023262C29383D373210151F1A0B0E040157
:1051600003060C09181D171230353F3A2B2E242147
:1051700060656F6A7B7E747153565C59484D474237
:10518000C0C5CFCADBDED4D1F3F6FCF9E8EDE7E227
:10519000A3A6ACA9B8BDB7B290959F9A8B8E848117
:1051A00080858F8A9B9E9491B3B6BCB9A8ADA7A207
:1051B000E3E6ECE9F8FDF7F2D0D5DFDACBCEC4C1F7
:1051C00043464C49585D575270757F7A6B6E6461E7
:1051D00020252F2A3B3E343113161C19080D0702D7
:1051E00000002110422063308440A550C660E77063
:1051F000088129914AA16BB18CC1ADD1CEE1EFF10B
:105200003112100273325222B5529442F772D662B2
:10521000399318837BB35AA3BDD39CC3FFF3DEE35A
:105220006224433420040114E664C774A444855402
:105230006AA54BB528850995EEE5CFF5ACC58DD5AA
:105240005336722611163006D776F6669556B44652
:105250005BB77AA719973887DFF7FEE79DD7BCC7FA
:10526000C448E5588668A7784008611802282338A2
:10527000CCC9EDD98EE9AFF9488969990AA92BB94A
:10528000F55AD44AB77A966A711A500A333A122AF2
:10529000FDDBDCCBBFFB9EEB799B588B3BBB1AAB9A
:1052A000A66C877CE44CC55C222C033C600C411C42
:1052B000AEED8FFDECCDCDDD2AAD0BBD688D499DEA
:1052C000977EB66ED55EF44E133E322E511E700E92
:1052D0009FFFBEEFDDDFFCCF1BBF3AAF599F788F3A
:1052E0008891A981CAB1EBA10CD12DC14EF16FE11A
:1052F0008010A100C230E320045025404670676052
:10530000B9839893FBA3DAB33DC31CD37FE35EF369
:10531000B1029012F322D2323542145277625672A1
:10532000EAB5CBA5A89589856EF54FE52CD50DC5B9
:10533000E234C324A01481046674476424540544F1
:10534000DBA7FAB79987B8975FE77EF71DC73CD709
:10535000D326F2369106B016576676761546345641
:105360004CD96DC90EF92FE9C899E9898AB9ABA959
:105370004458654806782768C018E1088238A32891
:105380007DCB5CDB3FEB1EFBF98BD89BBBAB9ABBA9
:10539000754A545A376A167AF10AD01AB32A923AE1
:1053A0002EFD0FED6CDD4DCDAABD8BADE89DC98DF9
:1053B000267C076C645C454CA23C832CE01CC10C31
:1053C0001FEF3EFF5DCF7CDF9BAFBABFD98FF89F49
:1053D000176E367E554E745E932EB23ED10EF01E81
:1053E000005EBCE2613FDD83C29C7E20A3FD1F41C5
:1053F0009DC3217FFCA2401E5F01E3BD3E6082DCB5
:10540000237D9FC1421CFEA0E1BF5D0380DE3C62A4
:10541000BEE0025CDF81633D7C22C09E1D43A1FF94
:105420004618FAA427799BC584DA3866E5BB590784
:10543000DB856739BAE406581947A5FB7826C49A74
:10544000653BD987045AB8E6A7F91B45C6987A2464
:10545000F8A6441A99C7257B3A6486D85B05E7B954
:105460008CD2306EEDB3510F4E10F2AC2F7193CD44
:10547000114FADF3702ECC92D38D6F31B2EC0E5034
:10548000AFF1134DCE90722C6D33D18F0C52B0EE24
:10549000326C8ED0530DEFB1F0AE4C1291CF2D7314
:1054A000CA947628ABF517490856B4EA6937D58B04
:1054B0005709EBB536688AD495CB2977F4AA4816F4
:1054C000E9B7550B88D6346A2B7597C94A14F6A8E4
:1054D000742AC896154BA9F7B6E80A54D7896B35D4
:1054E000EB3C904D53444F53352E300002020100E7
:1054F0000110000004F80C00010001000000000091
:1055000000000000000029EFBEADDE41544F4C20EA
:10551000465072696E74464154313220202000009A
:10552000000000000010000000200000003000001B
:10553000004000000050000000600000007000000B
:10554000008000000090000000A0000000B00000FB
:1055500000C0000000D0000000E0000000F00000EB
:105560000000010000800100000002000080020035
:10557000000003000080030000000400008004001D
:105580000000050000800500000006000080060005
:105590000000070000800700FF0F0000FF1F000051
:1055A000FF2F0000FF3F0000FF4F0000FF5F0000E3
:1055B000FF6F0000FF7F0000FF8F0000FF9F0000D3
:1055C000FFAF0000FFBF0000FFCF0000FFDF0000C3
:1055D000FFEF0000FFFF0000FF7F0100FFFF010061
:1055E000FF7F0200FFFF0200FF7F0300FFFF0300B9
:1055F000FF7F0400FFFF0400FF7F0500FFFF0500A1
:10560000FF7F0600FFFF0600FF7F0700FFFF070088
:10561000120110010000004051C2031300010420D8
:105620004801090220000101008032090400000243
:10563000080650620705820240000007050202408A
:10564000000000040309041C03410054004F004CF7
:10565000002000200020002000200020002000204A
:10566000002000280346005000720069006E00749C
:1056700000200046006C00610073006800200020DC
:1056800000200020002000200020001A03460069AE
:105690000072006D0077006100720065003000301C
:1056A00000300030000E034D0065006D006F007289
:1056B00000790000F122000000000000D702000085
:1056C00000000000000000000000000000000000DA
:1056D00000000000000000000000000000000000CA
:1056E00000000000000000000000000000000000BA
:1056F00000000000C5470000C5470000C947000082
:10570000DF470000C9470000DF470000DF47000017
:10571000DF470000F5470000C5470000C54700000F
:10572000C9470000DF470000C9470000DF4700000D
:10573000DF470000DF470000F5470000833E000020
:10574000893E0000733C0000833D0000B939000031
:10575000ED390000A1350000C33A00008F3E000083
:10576000BB2F0000C12F0000BD2A0000833D0000B8
:10577000B9390000172D0000C34200000B2E0000B5
:10578000C72F0000D7460000DD460000733C000034
:10579000833D0000B939000053440000C3420000BB
:1057A000294500008F3E00000000000000000000BE
:1057B00000000000000000000000000000000000E9
:1057C000000000000000000000000000EC57000096
:1057D000000000101C010000080100000859000032
:1057E0001C0100109C6C00002401000041544F4C2F
:1057F00020465072696E742800000000000000000E
:105800000000D4284B3D0000000000000000000014
:105810000000000000000000000000000000000088
:105820000000000000000000000000000000000078
:105830000000000000000000000000000000000068
:105840000000000000000000000000000000001048
:105850000000000000000000000000000000000048
:105860000000000000000000000000000000000038
:105870000000000000000000000000000000000028
:105880000000000000000000000000000000000018
:105890000000000000000000000000000000000008
:1058A00000000000000000000000000000000000F8
:1058B00000000000000000000000000000000000E8
:1058C0000000000000093D00000000000000000092
:1058D00000000000000000000000000000000000C8
:1058E00000000000000000000000000000000000B8
:1058F00000000000000000000000000000000000A8
:105900000000000000000000259213178551FE05DD
:105910000078B32A19DE8CF9A5A5C91DD7D4429405
:105920002CDE32D54AC9DB62EABF804F73508EB697
:10593000112153F687EF9E09FFB007E5CDED11CF9A
:1059400090FC5039981CB5B9E2ABE33233F5767A66
:1059500073381FEA3618A796A97A5555B5976894F3
:10596000CFB521310487D9288FABEA6092D21F9539
:105970000C2D92493F83EEB31172C824E32E19FA1D
:10598000252B5935A2D3C73C2AF3EE3BF068654975
:105990006309227DEED0D5EC4FD61E6210D2E96E9F
:1059A0000143FE22D22801BE8E18715E65FAC71A25
:1059B000AD0F73DBB8E7354ADE4C0357FF537FFE6C
:1059C000B8F0621B277868F837135FDBB8FBA6E7EF
:1059D000EFAEDA236C777F39C81250FC443C26EED8
:1059E000FCDC9D6E293E972264BF0E95F9E2900F74
:1059F000F239A07EAFDC95E9343320AAB69238D5CF
:105A00008AD490449EC32AD86462F22C9542511ED7
:105A1000EAACDBCC16227274F58AC000E31E037C6C
:105A20009C0DA01029FC8D3D585C00A9006A26E859
:105A300082132542FEAA0D40F6D0137CADAF0B4574
:105A40007F3FE4E234C5C946214929270AF008A965
:105A50009C6E63F6157595A076D7973CB75932D4EE
:105A6000237462A8F2C0EB6E6F9FDA021C1C8E6B6F
:105A7000C09BBB9C025A63FE9C1CB0912A79C7ACA8
:105A8000BD7D3806D677607CCEA9AD65D7408BB991
:105A9000FDE00A31CC89755AF7D0863B713BC6F8D8
:105AA00072CCAEB2A4DD04C03086AAE618B44D9123
:105AB000FB065EAEBED64137ED0248EE8655BD41CF
:105AC0005F0DB6A037DDF3D6AB1A99354CC9E3C7E5
:105AD000D64EFC6E502FA02D829E3FBFFE73A21E9D
:105AE000C0B01412D9F7B23E9BFA10211D183338FA
:105AF00085C2A0E927880049BE4F2823424163A000
:105B00002DEC5E50FA96A43B77A946CF2A69A7CB25
:105B1000DFDFBE0C1E2088882C54ACEFC8AAECE650
:105B20000E728EC9754B5B2A62F6542FC9D29F87BD
:105B3000961E1CBDA18933B203C52223A9E9F1D168
:105B4000C8004C8E852A8E00708349835A1DABF69F
:105B50002F31D4A85DDA6778C5000B38EB1062EFFF
:105B6000CED2424D2D855DE91AC5C1844AAEC834F6
:105B70008C3B062E0B4BA7A747F2BE3DF09510C4F9
:105B80000EBF66EDDC884CEABFF23A67BE46169C53
:105B9000CFED0EA5C6A1EB9C3FD5288F4DD93A403D
:105BA0004B294BD664C19D93F455CBDBBD1DB54548
:105BB000F8E83AE9C52752373CFA8B57A9AA7A0484
:105BC0002BDC498C2D988079E28FD9EEA830B4D0A7
:105BD00007FF593788552FBF916DBCEACC8BCBE4BA
:105BE000CA98C1C004A8739E6C8B4F12EB79B0A603
:105BF000A10C1D9025A411ECC754A5BDEE5AD7B237
:105C00002826D016B661680BFDDA2046EA624F7985
:105C1000425B381DA5738F66CA4F4A89099325B721
:105C2000506166AFFB64F8A51FA1B37B1441E8C4C3
:105C30003DCE6757D336F08D2AF02EF22A7C6E3F88
:105C4000FFEE6783580AD233164FEDD80493893696
:105C5000CB910B5BA8004E206A97AAB7658DCBCD80
:105C6000DB71A5775488D6F5DDA5D9203D5F81ADE0
:105C7000A81DDAA0690835E267475DF32B15E38CB0
:105C80006972378A049969994A0F0B15CB53CCB7BF
:105C9000A1D3B6F964B597CF5FFB4E18EBC2AE8BBC
:105CA000D5FE2AA34A0A6828F22CE3F84B81DF05C7
:105CB00037CEF36727548C5B8C055CFAB41891746B
:105CC0007EFF50AC81F65D5846DE9DE99CED574A5B
:105CD00010585D53F21398CC70AD9B0DC0CE981840
:105CE0000240946A89DFC0EBCD3A14DC1D3D7F0F82
:105CF000B11A25D932F3D919758E868D1CF084BC62
:105D000013D44A2D01ECB96A1E153643295D088C5F
:105D1000B58A41F69C95B0132250F9B298F3956874
:105D2000864FFE4E3EF33E73B77924114C1D4BFE59
:105D30002D6309745EA74FF3092C083ED38188F8C0
:105D400055A5B5603D300E61F8F460DAAFEFDD0EB9
:105D500070829EF5CB520E0B172249557C7BD21ACE
:105D60008ACBCD2AB905D3F31C3529EEB1386B0D9A
:105D7000713E223DF788CBB137002EFFB34CAC7398
:105D80007169131EC0BC4D6D2616897CE5B17C3946
:105D9000B04F8DF2B00FECC6F3982D4DF1555E3E2D
:105DA0009C72807916DD7FC39646DCA3380A0FCF3C
:105DB0002B8DEB9277848A716647463561F6BEFE7D
:105DC0006CCB2385028FAF098B32FCAAF527F4191F
:105DD000AF4976CFC24BF9DF8EB40CB9E5DDD63FC3
:105DE000408CEA14CBBA7BEF82AC54E6F117F14653
:105DF00038B775C52A1F5B0B0ACF8B06A2B2BAA3B0
:105E00009AD17A76390576CF09625736606759F6A6
:105E10006786668AB6DE1C7297382D68AD04A46F5B
:105E2000CBEDD71A2CF4B323D86592B6CF74423891
:105E300073B2A6C44CB61F22B027E24BA98AF0FC6D
:105E4000974BEE94EFD6D9014CBD77DAA494FD724E
:105E50003900DB9D70A8CFEA6DBBAA50E36CA42B80
:105E6000A1635B076EEB05D79480D90EEC048CF52B
:105E70009A70966D737BAB20BDC3B716A60C6F4AA4
:105E8000D1BFD2E2CB57224D89ABA13FE9EF84814C
:105E9000BE17F32EE47216AB14E06285E6B33353FB
:105EA000D0DF30249E6C36B37AAB839526740F9185
:105EB000627BA8BF064C16B06A340153D3CDF7A855
:105EC00027AF3D6DE43AAC51F9627D631E99803D88
:105ED000B926DF5375074CC4FE48C4DD123AB4D965
:105EE000AEC83386B8BB41B08ADDAB9AA832F51292
:105EF0000D2A07F080B19EBF6CC48202D41BDB4820
:105F0000ECCB2393DF481709FBEEB0206C6D958036
:105F100090649CE4245FE2B2E2AD5B009AF30BABC9
:105F2000A479234B0150183479EE31A7302A05EDBE
:105F30005B3557F2312968704A656FF1C092BFE155
:105F40004B4769C7B0FD2E3DF1302D34756F6CF7AE
:105F5000DCEFC671253F35E93D09D742A1BFA2A2BA
:105F600034B3913FA694AE6648E32D72EBF5854DB0
:105F7000C5F4407C9F0F49FD7AEEF19634B7640D6D
:105F80007A794230F1702A0AE7F9057929054A55EC
:105F900076B42DFCF935BD3CB6DE390EF02A3584D9
:105FA00022D5FAE3A29AAA83973DEFAA36A6A19A30
:105FB000E781950FD332BF60B5C238679D20AE3AF6
:105FC000FA5193D4FA605DB9E2A7AD48ADEF7CFF1A
:105FD0007187AC573F83BACF1EF86A8A19EB5DCC44
:105FE000A5D15F5206C6E79EE27463AA75B3EBE9DA
:105FF00039278020C522F14B579F8B3AA80F53B009
:00000001FF
